:0300000002116F7B
:03000B000200A54B
:03002B000202AE20
:03005B0002045F3D
:030073000204394B
:1000800002030406080C10182030406080040608A3
:100090000C10182030406080A0C00D0D0403060D28
:1000A0000503030202C2AFC0D0C0E020620C20688A
:1000B00002419D306602415DE47385258AC262E596
:1000C00025F4700221242068022111207210758B02
:1000D00000D0E0D0D0D292D291D290D2AF32D29290
:1000E000D291D2907406D5E0FDE53C1420E21520B3
:1000F000E10D207D02D295307D02D293020121D202
:1001000094020121207D02D293307D02D29502011A
:1001100021758B00D0E0D0D0D292D291D290D2AFC4
:1001200032758B00D0E0D0D0D2AF32419DE5256052
:100130000A207D02C292307D02C290D291419DE59B
:10014000256002C291207D02D290307D02D2924180
:100150009DE525600A207D02C290307D02C292207A
:100160007D02D292307D02D290419D207D02C293C9
:10017000307D02C295207D02C295307D02C293740B
:1001800006D5E0FDE525600A207D02C292307D02A1
:10019000C290D291419D207D02C293307D02C295D2
:1001A000C2947406D5E0FDE525600A207D02C29266
:1001B000307D02C290D291419DC294207D02C293B3
:1001C000307D02C2957406D5E0FDE5256002C2913E
:1001D000207D02D290307D02D292419DC294207D3A
:1001E00002C295307D02C2937406D5E0FDE525601C
:1001F00002C291207D02D290307D02D292419D2098
:100200007D02C295307D02C293C2947406D5E0FD92
:10021000E525600A207D02C290307D02C292207DD9
:1002200002D292307D02D290419D207D02C2953053
:100230007D02C293207D02C293307D02C295740676
:10024000D5E0FDE525600A207D02C290307D02C226
:1002500092207D02D292307D02D290419D30723D3B
:10026000E53C20E21A20E129207D02C293307D0284
:10027000C295207D02C295307D02C29302029D206C
:10028000E1E6207D02C293307D02C295C294020253
:100290009DC294207D02C295307D02C293E525F473
:1002A000F58A758B00D262D0E0D0D0D2AF32C2AF27
:1002B000C2AD53E6EFC0D0C0E0D2D3D2AFC2CEE5DC
:1002C0002960072074461529610C78007900E580C3
:1002D000307E01F430E40278FF53DACF207E03430E
:1002E000DA20307E0343DA10C2D8C271E580307E56
:1002F00001F430E40279FFC3E89970CE30610375F0
:1003000029402074037529408859D270E52A600479
:10031000152A611C20740543DA01C2D820700261DD
:1003200044A859206102C270207402612D882230D5
:10033000690AC3E522955E4003855E227882B60491
:1003400003852224C3E52594404002D26420CF0CCB
:10035000D0E0D0D0C2D343E610D2AD32C2CF7802C3
:10036000E52960053074021529C3E559940140055B
:10037000755C006186755D00756400E55C2401F5BF
:100380005C5003755CFF7982B7020EE547601EC3BF
:10039000E522943240178546227982B7030FE5475C
:1003A000600BC3E52294324004798E8722C3E52393
:1003B000952260084004152361BC0523D8C8056454
:1003C000E56470021564D565647565017805C3E55B
:1003D0006495664058C3E564956750087801756573
:1003E000030203F0C3E56495685005780175650163
:1003F000C3E55F9524401F7982B704028122E54757
:10040000701485245FE56404600385666475650186
:1004100075233C02042DE55F285005755FFF81229E
:10042000F55FE55F047006755DFF7564FFD0E0D091
:10043000D0C2D343E610D2AD32C0D0C0E0C2AF5379
:10044000917F53E67FC260759100C3E49550F594A7
:10045000E49551F595759104D0E0D0D0D2AF32C279
:10046000AF53E6EFC2ADC0D0C0E0C0F0D2D3D2AF40
:0E047000A8FBA9FCC2D830710281C653DACFB6
:10047E00207E0343DA10307E0343DA20D271E5800A
:10048E00307E01F420E402819D88268927C19D5388
:10049E00DACF207E0343DA20307E0343DA10C2D84F
:1004AE00C271307402C1897800E580307E01F4306B
:1004BE00E402C1898859C17053DACF207E0343DA32
:1004CE0020307E0343DA10C271206102A19653DA06
:1004DE00CF207E0343DA10307E0343DA20C2D8D217
:1004EE007188548955C3E89552F8E99553F9E4FBA0
:1004FE007E027A00C3E8948CE9940050057558008A
:10050E00A186C3E894C8E994005008E4D2E4FB7ACB
:10051E000AA163C3E89468E994015008E4D2E3FBAE
:10052E007A0FA163C3E894D0E994025008E4D2E2B2
:10053E00FB7A1EA163C3E894A0E994055008E4D2A7
:10054E00E1FB7A3CA163C3E89498E994085008E46F
:10055E00D2E0FB7A787E00C3E89556FCE99557FD0C
:10056E0030E708ECF42401FCEDF4FD755800C3EC03
:10057E009AED9E500375580188568957A854A9556F
:10058E00885289537802C170C3E89526F8E99527F9
:10059E00F9307C02C154307B02C154307A02C14D15
:1005AE00207502A1B9E9FDE8FCA1D8E9C313F9E869
:1005BE0013F8307902C14DE9C313F9E813F8307816
:1005CE0002C14DE9C313FDE813FC206126C3EC9470
:1005DE001CED94024002A1EFED7018C3EC94C850CC
:1005EE00120528C3E528940A5002C189755900D214
:1005FE0070C189E528600215287400207F03789663
:10060E00E624FAFEE43400FFC3EC9EFCED9FFD50A1
:10061E000678007900C154C3EC94FFED94004006B7
:10062E0078FF7900C154EC856FF0A4C5F0A2F733C2
:10063E00F87900400302067078FF7900020670E92F
:10064E00C313F9E813F8307C0EE9600278FFC3E8B3
:10065E001338F8E43400F9C3E894FFE9940040023B
:10066E0078FF8859D270206102C189741FF4552F0A
:10067E004BF52FC274E42B7002D27475294030747E
:10068E000375290A306102C19D20740353DAFE7589
:10069E002A20307403752A0AD0F0D0E0D0D0C2D30D
:1006AE00D2AD43E6103279010206D279030206D2A8
:1006BE00790A0206D2791E0206D279640206D2792E
:1006CE00C80206D27817E4D5E0FDD8FAD9F6227A18
:1006DE00147B780206F97A107B8C0206F97A0D7B70
:1006EE00B40206F97A0B7BC80206F9AC2575250112
:1006FE007902B27DE4C294D5E0FDE5256002C29197
:10070E00D5E0FDD291D5E0FDD294D5E0FDE5256092
:10071E000A207D02C292307D02C290E570D5E0FDC6
:10072E00207D02D292307D02D2907496D5E0FDD912
:10073E00C1EAF8D5E0FDD8FBDBB1C2948C2522C30B
:10074E007C007D0075F00005F0EA33FAEB33FB50C8
:10075E00F6EB13FBEA13FAC3E9FFE8FEE89AF8E9B1
:10076E009BF95004EFF9EEF8B3EC33FCED33FDD505
:10077E00F0DFEDF9ECF822E889F08A20D2D4F8A95E
:10078E00F07B0030F70B7BFFF42401F8E9F4340022
:10079E00F9E88520F0A4ADF0F8E98520F0A4AFF0DB
:1007AE00FEED2EF974003FFA7C04C3EA13FAE91346
:1007BE00F9E813F8DCF48BF030F70AE8F42401F8CA
:1007CE00E9F43400F9E889F0C2D4F8A9F02278826D
:1007DE00B6040302087EC3E5599419401FE52D5453
:1007EE00067019E547703878057994E71460077834
:1007FE000A1460027812C3E53B984020E547600971
:10080E0085615F7564FF756501852224E4F53EF50B
:10081E003FF540F541F542F54702087E75470179EF
:10082E0094E7147013E523F43333F913F8E9540104
:10083E0004F9E854FE020872E714147014E523F468
:10084E00333333F913F8E9540304F9E854FC02087E
:10085E007AE523F433333333F913F8E954070404F8
:0E086E00F9E854F8C39440F8E99400F9883E84
:10087C00893F22E547603BC3E53B13F9E53A13F8A2
:10088C00C3E53E98F8E53F99F9500CC3E89480E92C
:10089C0094FF40160208BAC3E8947FE99400500311
:1008AC000208BA787F79000208BA788079FF884309
:1008BC00894422E5476058E5432540F8E544354135
:1008CC00F9854420E4300701F43542FA30E709C3D6
:1008DC00EA94F040150208FCC3EA940F5003020896
:1008EC00FC78FF79FF7A0F0208FC780079007AF027
:1008FC00C3E524955E5006E52460092115E54420E6
:10090C00E70D2115E54430E706884089418A4222EB
:10091C00E547700302098078A1E6FAC3E54333F892
:10092C00E54433F9120785E930E70BC3E89480E915
:10093C0094FF40132157C3E8947FE994005002219F
:10094C0057787F79002157788079FFE820E715C325
:10095C00E52398F84009C3E89401400302097E7826
:10096C000102097EE8F424012523F8400302097EE4
:10097C0078FF884522E54770030209E378A2E6FA7E
:10098C00A841A942120785E930E70CC3E89401E9B4
:10099C0094FF40160209BAC3E894FFE9940050038F
:1009AC000209BA78FF79000209BA780179FFE920C7
:1009BC00E715C3E54598F84009C3E89401400302E4
:1009CC0009E178000209E1E8F424012545F8400327
:1009DC000209E178FF88242278FFC264E52D5406D1
:1009EC00702FD264C3E53B940A4009C3E5259440BB
:1009FC005002C264E53B601974FF853BF084853777
:100A0C00F0A4F8C5F0600278FFC3E895615002A825
:100A1C00618860227883E6F520120F7575E89012D4
:100A2C0006B475E890E5E820ECFBA8BDA9BE121051
:100A3C000D756BAF756C00C3740013FD74AF13FCB4
:100A4C0074AF2CFC74003DFDECFAEDFBC3E89AE9A5
:100A5C009B4014E56B24AFF56BE56C3400F56CEA48
:100A6C002CFAEB3DFB80E5AE6BAF6CC3E56C13F978
:100A7C00E56B13F8C3E913F9E813F8E56B28F5698E
:100A8C00E56C39F56A7A03C3E913F9E813F8DAF778
:100A9C00AA201A7009756B00756C00020ABA1AEA62
:100AAC006008EE28FEEF39FFDAF88E6B8F6C22753A
:100ABC00E890227883E6FFE5E820ECF7A8BDA9BE14
:100ACC00056DC3E56D94084052756D00E9FA79A087
:100ADC00E76044EA7007E56E601B020AF5C3E8950F
:100AEC006E6010E56E5006600C14020B010460F988
:100AFC00020B01E56EF56EC39458401B755EC0C3C6
:100B0C0094044013755E80C39404400B755E40C31F
:100B1C0094044003755E0075BB0322EFC39401601F
:100B2C001BC3E894FFE994035012C3E8956BE99555
:100B3C006C5009E55E600C155E020B4FE55EF460CF
:100B4C0002055EA85EC3E524985002A824C3E8956C
:100B5C005F400AA85FE55FF46003855F5E8825E56A
:100B6C006DB4070375BB1022743279A387F0A4C54A
:100B7C00F0A2F733F8C3E8955E4002A85E8822889D
:100B8C00248825886122753A00753B7F2275C82020
:100B9C00A8CCA9CD75C824AA38AB3988388939C3F3
:100BAC00E89AF8E99BF9AA3AAB3BAC3AAD3B7E0428
:100BBC007F02C3EB940440021E1FC3EB9408400257
:100BCC001E1FC3ED13FDEC13FCDEF7C3EA9CFAEB1E
:100BDC009DFBEF6009C3E913F9E813F8DFF7EA2886
:100BEC00FAEB39FB8A3A8B3B400122753AFF753B95
:100BFC00FF2230600261FE854C50854D51D260431E
:100C0C00E680227892E6FFC3E535948240010FC35B
:100C1C00E53594A040010FC3EF940640027F057E9A
:100C2C00021E3072010EC3E53B940350060E0E30CB
:100C3C0072010EC3E53B940250060E0E3072010E8B
:100C4C00A93BA83A7A04C3E913F9E813F8DAF7C315
:100C5C00E89EF8E99400F94009C3E89402E994008D
:0F0C6C0050047802E4F9E9FBE8FAC3E913FDE864
:100C7B0013FC884C894DC3EF94036037EF20E00DD4
:100C8B00E82CF8E93DF9ECFAEDFB020CABE828F89F
:100C9B00E939F9C3E89402F8E99400F97A02E4FB24
:100CAB00C3EF9403400D8A4E8B4F884889498C4A79
:100CBB008D4B22884E894F8A488B498C4A8D4B220B
:100CCB0030600281CBD26043E680E52D540660276D
:100CDB00A83AA93BE53494085006E820E002A94D58
:100CEB00759100C3E498F594E499F595759104D248
:100CFB006053917F43E68022D265753D00752000DD
:100D0B00020D16D265753D00752040E52D54066029
:100D1B0002C265D2AF206005E53D60012278017A01
:100D2B0002C3E53B940540027802C3E53B940A40BD
:100D3B00027803C3E53B940F40027A0330690478D1
:100D4B001E7A01206007E53D6003D2AF22D2AF00CF
:100D5B0000C2AFC3E53BFB940F40027B0FEB0430AB
:100D6B0073012320620123F93069027982E58BC379
:100D7B009940D0053DEAFBE59BF45440B52004DBDC
:100D8B00F6A1B2206502A116C265759100AE3AAF0D
:100D9B003BC3E49EF594E49FF595759104D26053A3
:100DAB00917F43E680A116306502A116D895D2AF8C
:100DBB002230690B0534206016753400020DDA20E1
:100DCB00600D20650A206B071581158102162B22F9
:100DDB00A84EA94F75910053917FC3E498F594E405
:100DEB0099F595759104854850854951D26043E634
:100DFB00802278003064053065027801E53575F0A6
:100E0B0007A4F9E5F028F5F0E9A2F013A2F113A27B
:100E1B00F213F535C394785003753578C3E53595E2
:100E2B00364008D266D292D291D290306002C1364F
:100E3B00854A50854B51D26043E68022D2A0C2AF87
:100E4B00C293C294C29530720B9001FF7406D5E029
:100E5B00FD020E87E53B54F86022E525600A207DF4
:100E6B0002C292307D02C2907406D5E0FD207D0255
:100E7B00D292307D02D2907406D5E0FD207D02D255
:100E8B0093307D02D295759F10753C02021008C2FB
:100E9B00A0C2AF207D02D290307D02D29230721769
:100EAB009001DCC294207D02C295307D02C2937406
:100EBB0006D5E0FD020EC590013F306206E52560C8
:100ECB0002C291207D03759F20307D03759F0075B5
:100EDB003C03021008C2AFC293C294C29530720B8E
:100EEB009001B97406D5E0FD020F1EE53B54F86086
:100EFB0022E525600A207D02C290307D02C29274E9
:100F0B0006D5E0FD207D02D290307D02D292740690
:100F1B00D5E0FD207D02D295307D02D293207D035A
:100F2B00759F00307D03759F20753C04021008C22D
:100F3B00AFD291307217900196207D02C293307D13
:100F4B0002C295C2947406D5E0FD020F5B90012D91
:100F5B0030620EE525600A207D02C292307D02C20E
:100F6B0090759F10753C05021008C2AFC293C294D6
:100F7B00C29530720B90016B7406D5E0FD020FA386
:100F8B00E53B54F86012E5256002C2917406D5E08A
:100F9B00FDD2917406D5E0FDD294207D03759F2080
:100FAB00307D03759F00753C06021008C2AF207D93
:100FBB0002D292307D02D29030721F90022A207D95
:100FCB0002C293307D02C295207D02C295307D0214
:100FDB00C2937406D5E0FD020FE890015130620E0A
:100FEB00E525600A207D02C290307D02C292207DF1
:100FFB0003759F00307D03759F20753C01C266D23F
:10100B00AF2290012BD292D291D290C293C294C2B2
:10101B0095C26222788076070876070876010876F3
:10102B00040876FF0876FF08760A08760208760130
:10103B00087601788C76010876000876B40876FF7E
:10104B000876FF0876FF0876030876FF0876010816
:10105B0076FF0876250876D00876780876C8087665
:0E106B00040876FF08760108760008767A08F9
:10107900760A087601227887E6FFC272BF0302D298
:10108900727888C27DE630E102D27DC27E7889E637
:1010990030E102D27EC3EF94026008758E01D273EB
:1010A9000210B1758E00C273227880E61490008018
:1010B9009378A1F67881E6149000809378A2F611CE
:1010C9000D227886E61490008D9378A3F6110D22EF
:1010D900789FE6F8700108C3E8941140027811E896
:1010E9002828F5662566256628F56725662828F5E2
:1010F9006822789CE67536FF75370CB4020675369A
:10110900A075370AB4030675368275370522227829
:1011190096E6FA7897E6FB307F047A007BFFC3EB0B
:101129009AFCC3948250027C82756F00056FEC852E
:101139006FF0A4C3E5F0948040F222D27F311812F7
:1011490006C37A007B007C101206B9E5592AFA74A5
:10115900003BFBDCF37C04C3EB13FBEA13FADCF77B
:10116900FEC27F311822E5EF20E603752000052035
:10117900903FFFE520146006901DFF146000930462
:10118900600375EF12C2D353D9BF7581C043FF8085
:101199001206B475EF0243B203E5B3240420E70253
:1011A900F5B3110D7580FF75A40075F1D475D4EFF1
:1011B90075908775A54075F2FF75D5BF75A6017540
:1011C900E24275DB4675EA02111F121664789886A9
:1011D90070C2AF1206CD1206DD1206C31206E41262
:1011E90006C31206EB1206C31217861206CD1206A3
:1011F900CD1206C8C2AFE4F8F6D8FD78C879C83070
:101209008407D9FBD8F7021C00111F121664117F3D
:1012190011B211CB11D911FB311731187898867099
:10122900110D75885075891275C82475910475D882
:101239004075A82275B80275E690759B80759D006A
:1012490075D10E75BC5875BB0375BA1175E8801256
:1012590006B4D2AF120A2043DA01C2D8C27112060B
:10126900CD753001D2617B037A0CE55870067A0C92
:10127900DB0221FD1206C320700221FDC270E5596F
:10128900C3940240E3E52F541F855B5AF55BB55AB9
:10129900D7DAD7C26153DACF207E0343DA20307E12
:1012A9000343DA10C2D8C271C2757528001206C884
:1012B900307409C3E528940A4002D2751206B97838
:1012C900023074027800C3E5599840F0C2AF1206A3
:1012D900DD1206DD1206DDD2AF1206CD754600120B
:1012E90006B9788CE6C3940150030213BCE530C3F8
:1012F900940150030213BC207435C3E55994FF507F
:10130900030213BCC2AF1206F2D2AF1206C8C3E57C
:1013190059940150EFC2AF1206DD1206BE1206DD66
:10132900D2AF1206C8C3E55994FF40E902180B7FF2
:1013390005D27F31181206C8C2AFC27F3118AE5923
:10134900C3E559947FD2AF40741206B4C2AF1206F6
:10135900F2D2AFDFDC3144C3EE94057897F612067A
:10136900CD1216A512178E7F0AD27F31181206C820
:10137900C2AFC27F3118AE59C3E559947FD2AF507D
:10138900E61206B4C2AF1206DD1206BE1206DDD29F
:10139900AFDFD63144EE24057896F61206CD121643
:1013A900A51217BD1206C83118C3E55994FF40F4B8
:1013B90002180BC3E559954640038559461206C8DC
:1013C90078017988E7B403027805C3E559984002A2
:1013D90041E8C2AF1206F21206F21206F2D2AF12B9
:1013E90006CD753000E4F531F5320531E531F4709B
:1013F900390532789AE67819146012783214600D3A
:10140900787D14600878FA146003753200C3E532F8
:1014190098401715327531B478998670C2AF1206A3
:10142900F2D2AF789886701206C81206BEE5297006
:101439000530740221FD78012074027806C3E5594C
:101449009840A71206C8E529700221FDC2AF110D07
:10145900E4F522F523F524F525D2AF78858662F5E2
:0F1469003EF53FF540F541F542F56DF547F52CA1
:10147800F52DF535120B92756D0875BB101206B473
:10148800120ABBE5E820ECFBA8BDA9BEE97001F88B
:10149800886E120ABF756D0875BB107887E6FE76F0
:1014A80002117F7887EEF6C2AF755EFF120B748566
:1014B800225E85225F852260D2AF752201752401E4
:1014C800752501855D64756501D268D2697534003A
:1014D800120F75120FB7120B92120B99120C0F0202
:1014E80014F4110D117F756D0075BB03120D0E12EA
:1014F8000DBC120DDB1207DC120DFD120E47120B8C
:1015080099120BFE120C0F120CCB120D03120DBC0C
:10151800120DDB12087F1209E4120DFD120E9A1249
:101528000B99120BFE120C0F120CCB120D0E120D92
:10153800BC120DDB1208BF120DFD120EE0120B9942
:10154800120BFE120C0F120CCB120D03120DBC1253
:101558000DDB12091C120DFD120F3A120B99120B1A
:10156800FE120C0F120CCB120D0E120DBC120DDB5D
:10157800120981120DFD120F75120B99120BFE1232
:101588000C0F120CCB120D03120ABB120DBC120D5C
:10159800DB120ABF120DFD120FB7120B99120BFEC8
:1015A800120C0F120CCB30692F206B2C85615E85D5
:1015B800615F855D6475650179327A0AC3E534999E
:1015C8004009C269D26A8A330215E0C3E559940119
:1015D80040030214F402162B306A1B206B18E53303
:1015E800147004C26A81EAF533C3E55994014003D3
:1015F8000214F402162BC3E55C9401400985615F6F
:10160800855D64756501C3E55C94FA501630740411
:10161800E529600FC3E53B78F0306B02786098509D
:101628000281F4C2AF110D7887E6FE7602117F7849
:1016380087EEF6E4F522F523F524F525F562C26870
:10164800D2AF1206B4110D307406E529700221FDDF
:10165800788DE6C39401400241C561EE901A0D7879
:10166800201216E7E520B4A50CA31216E7E520B46E
:101678005A03021685111F1216A50216A4901A0302
:1016880078807B0A1216E7A308DBF9901A0F788C8A
:101698007B151216E7A308DBF9901A2422C2AF12B1
:1016A8001726121700901A00740D1216ECA3740274
:1016B8001216ECA374131216EC901A0378807B0AA6
:1016C8001216EBA308DBF9901A0F788C7B1512160B
:1016D800EBA308DBF9121739121717901A2422E422
:1016E80093F622E6438F01538FFD75EF0275B7A578
:1016F80075B7F1F0538FFE22438F02438F0175EFC8
:101708000275B7A575B7F1901A0DF0538FFC2290AA
:101718001A0D74A5D1EC901A0E745AD1EC227A30B5
:1017280079D07820901A40D1E7E520F709A3DAF7B5
:10173800227A3079D0901A40E7D1EC09A3DAF9225D
:10174800AB71A872BB01027980BB02027981BB032D
:10175800027982BB04027994BB05027983BB060235
:101768007986BB07027992BB08027987BB0902799F
:101778009CBB0A027988BB0B027989E8F7227C05B1
:101788001206CDDCFB22C2AF1206DD1206E41206F9
:10179800EB1206F21206BE1206DD1206E41206EB82
:1017A8001206F21206BE1206DD1206E41206EB124B
:1017B80006F2D2AF22C2AF1206F21206EB1206E40C
:1017C8001206DD1206BE1206F21206EB1206E4122B
:1017D80006DD1206BE1206F21206EB1206E4120627
:1017E800DDD2AF22AE71AF72C2AF1206DD1206DDD6
:1017F8001206DD1206BEDEF21206F21206BEDFF88F
:10180800D2AF2212178E12178612178675710175BC
:1018180072017573001217EC7C05AD591206CDC321
:10182800ED955970F5C3E5599401400AC3E55994FB
:10183800FF403702184F1217481216A512178EC20A
:10184800AF75EF12121786DCD10573C3E5739403E5
:10185800500280C11217860572E5711490009A93A0
:0D186800F808C3E57298500280A812178698
:101875001217860571C3E571940C500280941210FD
:0C1885001F1216A5C2AF75EF12121786D5
:101A00000D021307070104FFFF0A020101A55A0195
:101A100000B4FFFFFF03FF01FF25D078C804FF01DA
:051A200000FF0A01FFB8
:101A400023484B696E67323041232020202020201C
:101A500023424C48454C4923463333302320202031
:101A60002020202020202020202020202020202076
:101C0000C2AFC2D353D9BF7581C043B20343FF8073
:101C1000752438752503B1BF75EF0275E24043F1B5
:101C20001053A4EFD284780379E67C1075220075F6
:101C30002300901DCC7B0675249875250130840205
:101C4000813D208408D8FBD9F9DCF781AD308408C8
:101C5000D8FBD9F9DCF781ADB17FE493A3C39A60D7
:101C6000028126DBDDB171600281267B08E493FAF4
:101C7000A3B152DBF87A30B152752200752300B15E
:101C800071EAFCEBFDC3ED94FE400EB1718A278B27
:101C900028ED30E0048A828B83B1717AC270D8C398
:101CA000ED94FE601050CEBD0022EC600675200061
:101CB0000200008100A827A9280809D804D90281B8
:101CC000C9B175EA89AAF281BB0D8199C3ED94036C
:101CD0005049EDA2E092007AC5C3E5829400E58305
:101CE000941C5093200010438F02438F0175B7A5B9
:101CF00075B7F1F030001FA827A9280809438F0104
:101D0000538FFDD804D902A11689AAE275B7A5752B
:101D1000B7F1F0A3A103538FFC81757AC1BD030C09
:101D2000E493A3FAB136DCF8B12E81758177AA224B
:101D3000AB23B152EBFAEA6222752608C3E52313FE
:101D4000F523E52213F52250066323A0632201D573
:101D500026EAB1BFB1BF75260AEAF4200102D28497
:101D6000300102C284B1BFC3134002C201D526EBC9
:101D700022B175EAFB208402A175308402A17A7534
:101D80002608AE24AF25C3EF13FFEE13FEB1C3B197
:101D9000BFC3EA133084024480FA30E703632201B0
:101DA000C3E52313F523E52213F52250066323A090
:101DB000632201D526D9E52265236523F52222AECB
:101DC00024AF250E0FDEFEDFFCD20122424C486517
:0A1DD0006C6934373132F33006013C
:00000001FF
